 rawmnntfy001

 Timestamp is 6090189f (reproducible build file hash)

 Preferred load address is 0000000180000000

 Start         Length     Name                   Class
 0001:00000000 00002fb0H .text$mn                CODE
 0001:00002fb0 00000036H .text$mn$00             CODE
 0001:00002fe6 00000092H .text$x                 CODE
 0002:00000000 00000198H .idata$5                DATA
 0002:00000198 00000038H .00cfg                  DATA
 0002:000001d0 00000008H .CRT$XCA                DATA
 0002:000001d8 00000008H .CRT$XCZ                DATA
 0002:000001e0 00000008H .CRT$XIA                DATA
 0002:000001e8 00000008H .CRT$XIC                DATA
 0002:000001f0 00000008H .CRT$XIZ                DATA
 0002:000001f8 00000008H .CRT$XLA                DATA
 0002:00000200 00000008H .CRT$XLZ                DATA
 0002:00000208 00000008H .CRT$XPA                DATA
 0002:00000210 00000008H .CRT$XPZ                DATA
 0002:00000218 00000008H .CRT$XTA                DATA
 0002:00000220 00000010H .CRT$XTZ                DATA
 0002:00000228 00000000H .gehcont$y              DATA
 0002:00000228 00000000H .gfids$y                DATA
 0002:00000230 00001bd0H .rdata                  DATA
 0002:00001e00 00000000H .rdata$CastGuardVftablesA DATA
 0002:00001e00 00000000H .rdata$CastGuardVftablesC DATA
 0002:00001e00 00000028H .rdata$T                DATA
 0002:00001e28 000000a4H .rdata$voltmd           DATA
 0002:00001ecc 0000031cH .rdata$zzzdbg           DATA
 0002:000021e8 00000008H .rtc$IAA                DATA
 0002:000021f0 00000008H .rtc$IZZ                DATA
 0002:000021f8 00000008H .rtc$TAA                DATA
 0002:00002200 00000008H .rtc$TZZ                DATA
 0002:00002208 00000004H .tls                    DATA
 0002:0000220c 00000004H .tls$                   DATA
 0002:00002210 00000008H .tls$ZZZ                DATA
 0002:00002218 00000308H .xdata                  DATA
 0002:00002520 000003a4H .edata                  DATA
 0002:000028c4 00000064H .idata$2                DATA
 0002:00002928 00000018H .idata$3                DATA
 0002:00002940 00000198H .idata$4                DATA
 0002:00002ad8 0000041eH .idata$6                DATA
 0003:00000000 00000080H .data                   DATA
 0003:00000080 0001d378H .bss                    DATA
 0004:00000000 00000390H .pdata                  DATA

  Address         Publics by Value              Rva+Base               Lib:Object

 0000:00000000       __AbsoluteZero             0000000000000000     <absolute>
 0000:00000000       ___safe_se_handler_count   0000000000000000     <absolute>
 0000:00000000       ___safe_se_handler_table   0000000000000000     <absolute>
 0000:00000000       __arm64x_extra_rfe_table   0000000000000000     <absolute>
 0000:00000000       __arm64x_extra_rfe_table_size 0000000000000000     <absolute>
 0000:00000000       __arm64x_native_entrypoint 0000000000000000     <absolute>
 0000:00000000       __arm64x_redirection_metadata 0000000000000000     <absolute>
 0000:00000000       __arm64x_redirection_metadata_count 0000000000000000     <absolute>
 0000:00000000       __dynamic_value_reloc_table 0000000000000000     <absolute>
 0000:00000000       __enclave_config           0000000000000000     <absolute>
 0000:00000000       __guard_check_icall_a64n_fptr 0000000000000000     <absolute>
 0000:00000000       __guard_eh_cont_count      0000000000000000     <absolute>
 0000:00000000       __guard_eh_cont_table      0000000000000000     <absolute>
 0000:00000000       __guard_fids_count         0000000000000000     <absolute>
 0000:00000000       __guard_fids_table         0000000000000000     <absolute>
 0000:00000000       __guard_iat_count          0000000000000000     <absolute>
 0000:00000000       __guard_iat_table          0000000000000000     <absolute>
 0000:00000000       __guard_longjmp_count      0000000000000000     <absolute>
 0000:00000000       __guard_longjmp_table      0000000000000000     <absolute>
 0000:00000000       __hybrid_auxiliary_iat     0000000000000000     <absolute>
 0000:00000000       __hybrid_auxiliary_iat_copy 0000000000000000     <absolute>
 0000:00000000       __hybrid_code_map          0000000000000000     <absolute>
 0000:00000000       __hybrid_code_map_count    0000000000000000     <absolute>
 0000:00000000       __x64_code_ranges_to_entry_points 0000000000000000     <absolute>
 0000:00000000       __x64_code_ranges_to_entry_points_count 0000000000000000     <absolute>
 0000:00000100       __guard_flags              0000000000000100     <absolute>
 0000:00000000       __ImageBase                0000000180000000     <linker-defined>
 0001:00000000       ?NewObject@JNIEnv_@@QEAAPEAV_jobject@@PEAV_jclass@@PEAU_jmethodID@@ZZ 0000000180001000 f i librawmnntfy001.obj
 0001:00000028       ?SetEventNotificationMode@_jvmtiEnv@@QEAA?AW4jvmtiError@@W4jvmtiEventMode@@W4jvmtiEvent@@PEAV_jobject@@ZZ 0000000180001028 f i librawmnntfy001.obj
 0001:00000034       ?TranslateError@@YAPEBDW4jvmtiError@@@Z 0000000180001034 f   librawmnntfy001.obj
 0001:000002ec       ?nsk_jni_check_exception@@YAHPEAUJNIEnv_@@QEBDH@Z 00000001800012ec f   librawmnntfy001.obj
 0001:00000430       ?nsk_jni_lverify@@YAHHPEAUJNIEnv_@@HQEBDH1ZZ 0000000180001430 f   librawmnntfy001.obj
 0001:000004d0       Agent_Initialize           00000001800014d0 f   librawmnntfy001.obj
 0001:000005cc       Agent_OnAttach             00000001800015cc f   librawmnntfy001.obj
 0001:000005cc       Agent_OnLoad               00000001800015cc f   librawmnntfy001.obj
 0001:000005d4       Java_nsk_jvmti_RawMonitorNotify_rawmnntfy001_check 00000001800015d4 f   librawmnntfy001.obj
 0001:00000868       Java_nsk_jvmti_unit_FollowReferences_FollowRefObjects_addRefToVerify 0000000180001868 f   librawmnntfy001.obj
 0001:00000a40       Java_nsk_jvmti_unit_FollowReferences_FollowRefObjects_getTag 0000000180001a40 f   librawmnntfy001.obj
 0001:00000b00       Java_nsk_jvmti_unit_FollowReferences_FollowRefObjects_resetRefsToVerify 0000000180001b00 f   librawmnntfy001.obj
 0001:00000b08       Java_nsk_jvmti_unit_FollowReferences_FollowRefObjects_resetTags 0000000180001b08 f   librawmnntfy001.obj
 0001:00000b4c       Java_nsk_jvmti_unit_FollowReferences_FollowRefObjects_setTag 0000000180001b4c f   librawmnntfy001.obj
 0001:00000da4       Java_nsk_share_jvmti_ArgumentHandler_getAgentOptionsString 0000000180001da4 f   librawmnntfy001.obj
 0001:00000e54       Java_nsk_share_jvmti_DebugeeClass_checkStatus 0000000180001e54 f   librawmnntfy001.obj
 0001:00000edc       Java_nsk_share_jvmti_DebugeeClass_resetAgentData 0000000180001edc f   librawmnntfy001.obj
 0001:00000f3c       Java_nsk_share_jvmti_RedefineAgent_agentStatus 0000000180001f3c f   librawmnntfy001.obj
 0001:00000f48       Java_nsk_share_jvmti_RedefineAgent_isRedefined 0000000180001f48 f   librawmnntfy001.obj
 0001:00000f54       Java_nsk_share_jvmti_RedefineAgent_redefineAttempted 0000000180001f54 f   librawmnntfy001.obj
 0001:00000f60       MA_checkStatus             0000000180001f60 f   librawmnntfy001.obj
 0001:00001004       VMInit                     0000000180002004 f   librawmnntfy001.obj
 0001:00001290       __local_stdio_printf_options 0000000180002290 f i librawmnntfy001.obj
 0001:00001298       _snprintf                  0000000180002298 f i librawmnntfy001.obj
 0001:000014c8       exitOnError                00000001800024c8 f   librawmnntfy001.obj
 0001:0000157c       fprintf                    000000018000257c f i librawmnntfy001.obj
 0001:000015c0       nsk_jvmti_lverify          00000001800025c0 f   librawmnntfy001.obj
 0001:000016b0       nsk_jvmti_resetAgentData   00000001800026b0 f   librawmnntfy001.obj
 0001:00001730       nsk_jvmti_setFailStatus    0000000180002730 f   librawmnntfy001.obj
 0001:0000176c       nsk_lcomplain              000000018000276c f   librawmnntfy001.obj
 0001:0000178c       nsk_ldisplay               000000018000278c f   librawmnntfy001.obj
 0001:000017ac       nsk_ltrace                 00000001800027ac f   librawmnntfy001.obj
 0001:000017cc       nsk_lvcomplain             00000001800027cc f   librawmnntfy001.obj
 0001:00001984       nsk_lvdisplay              0000000180002984 f   librawmnntfy001.obj
 0001:000019d0       nsk_lverify                00000001800029d0 f   librawmnntfy001.obj
 0001:00001a2c       nsk_lvtrace                0000000180002a2c f   librawmnntfy001.obj
 0001:00001a8c       nsk_printf                 0000000180002a8c f   librawmnntfy001.obj
 0001:00001ab4       nsk_vprintf                0000000180002ab4 f   librawmnntfy001.obj
 0001:00001b68       printf                     0000000180002b68 f i librawmnntfy001.obj
 0001:00002090       __raise_securityfailure    0000000180003090 f   MSVCRT:gs_report.obj
 0001:000020c4       __report_gsfailure         00000001800030c4 f   MSVCRT:gs_report.obj
 0001:00002304       __GSHandlerCheck           0000000180003304 f   MSVCRT:gshandler.obj
 0001:00002324       __GSHandlerCheckCommon     0000000180003324 f   MSVCRT:gshandler.obj
 0001:00002390       __security_check_cookie    0000000180003390 f   MSVCRT:amdsecgs.obj
 0001:000026d0       _DllMainCRTStartup         00000001800036d0 f   MSVCRT:dll_dllmain.obj
 0001:00002710       __scrt_acquire_startup_lock 0000000180003710 f   MSVCRT:utility.obj
 0001:0000274c       __scrt_dllmain_after_initialize_c 000000018000374c f   MSVCRT:utility.obj
 0001:00002780       __scrt_dllmain_before_initialize_c 0000000180003780 f   MSVCRT:utility.obj
 0001:00002798       __scrt_dllmain_crt_thread_attach 0000000180003798 f   MSVCRT:utility.obj
 0001:000027c0       __scrt_dllmain_crt_thread_detach 00000001800037c0 f   MSVCRT:utility.obj
 0001:000027d8       __scrt_dllmain_exception_filter 00000001800037d8 f   MSVCRT:utility.obj
 0001:00002838       __scrt_dllmain_uninitialize_c 0000000180003838 f   MSVCRT:utility.obj
 0001:00002868       __scrt_dllmain_uninitialize_critical 0000000180003868 f   MSVCRT:utility.obj
 0001:0000287c       __scrt_initialize_crt      000000018000387c f   MSVCRT:utility.obj
 0001:000028c8       __scrt_initialize_onexit_tables 00000001800038c8 f   MSVCRT:utility.obj
 0001:00002954       __scrt_is_nonwritable_in_current_image 0000000180003954 f   MSVCRT:utility.obj
 0001:000029ec       __scrt_release_startup_lock 00000001800039ec f   MSVCRT:utility.obj
 0001:00002a10       __scrt_uninitialize_crt    0000000180003a10 f   MSVCRT:utility.obj
 0001:00002a3c       _onexit                    0000000180003a3c f   MSVCRT:utility.obj
 0001:00002a78       atexit                     0000000180003a78 f   MSVCRT:utility.obj
 0001:00002a90       __crt_debugger_hook        0000000180003a90 f   MSVCRT:utility_desktop.obj
 0001:00002a98       __scrt_fastfail            0000000180003a98 f   MSVCRT:utility_desktop.obj
 0001:00002be4       _guard_check_icall_nop     0000000180003be4 f i MSVCRT:guard_support.obj
 0001:00002be8       __security_init_cookie     0000000180003be8 f   MSVCRT:gs_support.obj
 0001:00002c94       DllMain                    0000000180003c94 f   MSVCRT:dll_dllmain_stub.obj
 0001:00002cb8       ?__scrt_initialize_type_info@@YAXXZ 0000000180003cb8 f   MSVCRT:tncleanup.obj
 0001:00002cc8       ?__scrt_uninitialize_type_info@@YAXXZ 0000000180003cc8 f   MSVCRT:tncleanup.obj
 0001:00002cd4       __local_stdio_scanf_options 0000000180003cd4 f i MSVCRT:default_local_stdio_options.obj
 0001:00002cdc       __scrt_initialize_default_local_stdio_options 0000000180003cdc f   MSVCRT:default_local_stdio_options.obj
 0001:00002cf8       __scrt_get_dyn_tls_init_callback 0000000180003cf8 f   MSVCRT:dyn_tls_init.obj
 0001:00002d00       _RTC_Initialize            0000000180003d00 f   MSVCRT:initsect.obj
 0001:00002d3c       _RTC_Terminate             0000000180003d3c f   MSVCRT:initsect.obj
 0001:00002d78       __isa_available_init       0000000180003d78 f   MSVCRT:cpu_disp.obj
 0001:00002f24       _get_startup_argv_mode     0000000180003f24 f   MSVCRT:argv_mode.obj
 0001:00002f2c       __scrt_is_ucrt_dll_in_use  0000000180003f2c f   MSVCRT:ucrt_detection.obj
 0001:00002f40       memcpy                     0000000180003f40 f   vcruntime:VCRUNTIME140.dll
 0001:00002f46       memset                     0000000180003f46 f   vcruntime:VCRUNTIME140.dll
 0001:00002f4c       strchr                     0000000180003f4c f   vcruntime:VCRUNTIME140.dll
 0001:00002f52       __C_specific_handler       0000000180003f52 f   vcruntime:VCRUNTIME140.dll
 0001:00002f58       __std_type_info_destroy_list 0000000180003f58 f   vcruntime:VCRUNTIME140.dll
 0001:00002f5e       strcmp                     0000000180003f5e f   ucrt:api-ms-win-crt-string-l1-1-0.dll
 0001:00002f64       strlen                     0000000180003f64 f   ucrt:api-ms-win-crt-string-l1-1-0.dll
 0001:00002f6a       _initterm                  0000000180003f6a f   ucrt:api-ms-win-crt-runtime-l1-1-0.dll
 0001:00002f70       _initterm_e                0000000180003f70 f   ucrt:api-ms-win-crt-runtime-l1-1-0.dll
 0001:00002f76       _seh_filter_dll            0000000180003f76 f   ucrt:api-ms-win-crt-runtime-l1-1-0.dll
 0001:00002f7c       _configure_narrow_argv     0000000180003f7c f   ucrt:api-ms-win-crt-runtime-l1-1-0.dll
 0001:00002f82       _initialize_narrow_environment 0000000180003f82 f   ucrt:api-ms-win-crt-runtime-l1-1-0.dll
 0001:00002f88       _initialize_onexit_table   0000000180003f88 f   ucrt:api-ms-win-crt-runtime-l1-1-0.dll
 0001:00002f8e       _register_onexit_function  0000000180003f8e f   ucrt:api-ms-win-crt-runtime-l1-1-0.dll
 0001:00002f94       _execute_onexit_table      0000000180003f94 f   ucrt:api-ms-win-crt-runtime-l1-1-0.dll
 0001:00002f9a       _crt_atexit                0000000180003f9a f   ucrt:api-ms-win-crt-runtime-l1-1-0.dll
 0001:00002fa0       _cexit                     0000000180003fa0 f   ucrt:api-ms-win-crt-runtime-l1-1-0.dll
 0001:00002fa8       __acrt_initialize          0000000180003fa8 f   MSVCRT:ucrt_stubs.obj
 0001:00002fa8       __acrt_thread_attach       0000000180003fa8 f   MSVCRT:ucrt_stubs.obj
 0001:00002fa8       __acrt_thread_detach       0000000180003fa8 f   MSVCRT:ucrt_stubs.obj
 0001:00002fa8       __acrt_uninitialize        0000000180003fa8 f   MSVCRT:ucrt_stubs.obj
 0001:00002fa8       __acrt_uninitialize_critical 0000000180003fa8 f   MSVCRT:ucrt_stubs.obj
 0001:00002fa8       __scrt_stub_for_acrt_initialize 0000000180003fa8 f   MSVCRT:ucrt_stubs.obj
 0001:00002fa8       __scrt_stub_for_acrt_thread_attach 0000000180003fa8 f   MSVCRT:ucrt_stubs.obj
 0001:00002fa8       __scrt_stub_for_acrt_thread_detach 0000000180003fa8 f   MSVCRT:ucrt_stubs.obj
 0001:00002fa8       __scrt_stub_for_acrt_uninitialize 0000000180003fa8 f   MSVCRT:ucrt_stubs.obj
 0001:00002fa8       __scrt_stub_for_acrt_uninitialize_critical 0000000180003fa8 f   MSVCRT:ucrt_stubs.obj
 0001:00002fa8       __vcrt_initialize          0000000180003fa8 f   MSVCRT:ucrt_stubs.obj
 0001:00002fa8       __vcrt_thread_attach       0000000180003fa8 f   MSVCRT:ucrt_stubs.obj
 0001:00002fa8       __vcrt_thread_detach       0000000180003fa8 f   MSVCRT:ucrt_stubs.obj
 0001:00002fa8       __vcrt_uninitialize        0000000180003fa8 f   MSVCRT:ucrt_stubs.obj
 0001:00002fa8       __vcrt_uninitialize_critical 0000000180003fa8 f   MSVCRT:ucrt_stubs.obj
 0001:00002fac       __scrt_stub_for_is_c_termination_complete 0000000180003fac f   MSVCRT:ucrt_stubs.obj
 0001:00002fac       _is_c_termination_complete 0000000180003fac f   MSVCRT:ucrt_stubs.obj
 0001:00002fc0       _guard_dispatch_icall_nop  0000000180003fc0 f   MSVCRT:guard_dispatch.obj
 0001:00002fe0       _guard_xfg_dispatch_icall_nop 0000000180003fe0 f   MSVCRT:guard_xfg_dispatch.obj
 0002:00000000       __imp_RtlCaptureContext    0000000180005000     kernel32:KERNEL32.dll
 0002:00000008       __imp_RtlLookupFunctionEntry 0000000180005008     kernel32:KERNEL32.dll
 0002:00000010       __imp_RtlVirtualUnwind     0000000180005010     kernel32:KERNEL32.dll
 0002:00000018       __imp_UnhandledExceptionFilter 0000000180005018     kernel32:KERNEL32.dll
 0002:00000020       __imp_SetUnhandledExceptionFilter 0000000180005020     kernel32:KERNEL32.dll
 0002:00000028       __imp_GetCurrentProcess    0000000180005028     kernel32:KERNEL32.dll
 0002:00000030       __imp_TerminateProcess     0000000180005030     kernel32:KERNEL32.dll
 0002:00000038       __imp_IsProcessorFeaturePresent 0000000180005038     kernel32:KERNEL32.dll
 0002:00000040       __imp_CloseHandle          0000000180005040     kernel32:KERNEL32.dll
 0002:00000048       __imp_InitializeCriticalSectionAndSpinCount 0000000180005048     kernel32:KERNEL32.dll
 0002:00000050       __imp_DeleteCriticalSection 0000000180005050     kernel32:KERNEL32.dll
 0002:00000058       __imp_CreateEventW         0000000180005058     kernel32:KERNEL32.dll
 0002:00000060       __imp_GetModuleHandleW     0000000180005060     kernel32:KERNEL32.dll
 0002:00000068       __imp_GetProcAddress       0000000180005068     kernel32:KERNEL32.dll
 0002:00000070       __imp_IsDebuggerPresent    0000000180005070     kernel32:KERNEL32.dll
 0002:00000078       __imp_QueryPerformanceCounter 0000000180005078     kernel32:KERNEL32.dll
 0002:00000080       __imp_GetCurrentProcessId  0000000180005080     kernel32:KERNEL32.dll
 0002:00000088       __imp_GetCurrentThreadId   0000000180005088     kernel32:KERNEL32.dll
 0002:00000090       __imp_GetSystemTimeAsFileTime 0000000180005090     kernel32:KERNEL32.dll
 0002:00000098       __imp_DisableThreadLibraryCalls 0000000180005098     kernel32:KERNEL32.dll
 0002:000000a0       __imp_InitializeSListHead  00000001800050a0     kernel32:KERNEL32.dll
 0002:000000a8       \177KERNEL32_NULL_THUNK_DATA 00000001800050a8     kernel32:KERNEL32.dll
 0002:000000b0       __imp_memcpy               00000001800050b0     vcruntime:VCRUNTIME140.dll
 0002:000000b8       __imp_memset               00000001800050b8     vcruntime:VCRUNTIME140.dll
 0002:000000c0       __imp_strchr               00000001800050c0     vcruntime:VCRUNTIME140.dll
 0002:000000c8       __imp___C_specific_handler 00000001800050c8     vcruntime:VCRUNTIME140.dll
 0002:000000d0       __imp___std_type_info_destroy_list 00000001800050d0     vcruntime:VCRUNTIME140.dll
 0002:000000d8       \177VCRUNTIME140_NULL_THUNK_DATA 00000001800050d8     vcruntime:VCRUNTIME140.dll
 0002:000000e0       __imp__errno               00000001800050e0     ucrt:api-ms-win-crt-runtime-l1-1-0.dll
 0002:000000e8       __imp_exit                 00000001800050e8     ucrt:api-ms-win-crt-runtime-l1-1-0.dll
 0002:000000f0       __imp__cexit               00000001800050f0     ucrt:api-ms-win-crt-runtime-l1-1-0.dll
 0002:000000f8       __imp__crt_atexit          00000001800050f8     ucrt:api-ms-win-crt-runtime-l1-1-0.dll
 0002:00000100       __imp__execute_onexit_table 0000000180005100     ucrt:api-ms-win-crt-runtime-l1-1-0.dll
 0002:00000108       __imp__register_onexit_function 0000000180005108     ucrt:api-ms-win-crt-runtime-l1-1-0.dll
 0002:00000110       __imp__initialize_onexit_table 0000000180005110     ucrt:api-ms-win-crt-runtime-l1-1-0.dll
 0002:00000118       __imp__initialize_narrow_environment 0000000180005118     ucrt:api-ms-win-crt-runtime-l1-1-0.dll
 0002:00000120       __imp__configure_narrow_argv 0000000180005120     ucrt:api-ms-win-crt-runtime-l1-1-0.dll
 0002:00000128       __imp__seh_filter_dll      0000000180005128     ucrt:api-ms-win-crt-runtime-l1-1-0.dll
 0002:00000130       __imp__initterm_e          0000000180005130     ucrt:api-ms-win-crt-runtime-l1-1-0.dll
 0002:00000138       __imp__initterm            0000000180005138     ucrt:api-ms-win-crt-runtime-l1-1-0.dll
 0002:00000140       \177api-ms-win-crt-runtime-l1-1-0_NULL_THUNK_DATA 0000000180005140     ucrt:api-ms-win-crt-runtime-l1-1-0.dll
 0002:00000148       __imp___acrt_iob_func      0000000180005148     ucrt:api-ms-win-crt-stdio-l1-1-0.dll
 0002:00000150       __imp_fflush               0000000180005150     ucrt:api-ms-win-crt-stdio-l1-1-0.dll
 0002:00000158       __imp___stdio_common_vsprintf 0000000180005158     ucrt:api-ms-win-crt-stdio-l1-1-0.dll
 0002:00000160       __imp___stdio_common_vfprintf 0000000180005160     ucrt:api-ms-win-crt-stdio-l1-1-0.dll
 0002:00000168       \177api-ms-win-crt-stdio-l1-1-0_NULL_THUNK_DATA 0000000180005168     ucrt:api-ms-win-crt-stdio-l1-1-0.dll
 0002:00000170       __imp_strcmp               0000000180005170     ucrt:api-ms-win-crt-string-l1-1-0.dll
 0002:00000178       __imp__strdup              0000000180005178     ucrt:api-ms-win-crt-string-l1-1-0.dll
 0002:00000178       __imp_strdup               0000000180005178     ucrt:api-ms-win-crt-string-l1-1-0.dll
 0002:00000180       __imp_strlen               0000000180005180     ucrt:api-ms-win-crt-string-l1-1-0.dll
 0002:00000188       __imp_strncpy              0000000180005188     ucrt:api-ms-win-crt-string-l1-1-0.dll
 0002:00000190       \177api-ms-win-crt-string-l1-1-0_NULL_THUNK_DATA 0000000180005190     ucrt:api-ms-win-crt-string-l1-1-0.dll
 0002:00000198       __guard_check_icall_fptr   0000000180005198     MSVCRT:guard_support.obj
 0002:000001a0       __guard_xfg_check_icall_fptr 00000001800051a0     MSVCRT:guard_support.obj
 0002:000001a8       __guard_dispatch_icall_fptr 00000001800051a8     MSVCRT:guard_support.obj
 0002:000001b0       __guard_xfg_dispatch_icall_fptr 00000001800051b0     MSVCRT:guard_support.obj
 0002:000001b8       __guard_xfg_table_dispatch_icall_fptr 00000001800051b8     MSVCRT:guard_support.obj
 0002:000001c0       __castguard_check_failure_os_handled_fptr 00000001800051c0     MSVCRT:guard_support.obj
 0002:000001c8       __guard_memcpy_fptr        00000001800051c8     vcruntime:softmemtag.obj
 0002:000001d0       __xc_a                     00000001800051d0     MSVCRT:initializers.obj
 0002:000001d8       __xc_z                     00000001800051d8     MSVCRT:initializers.obj
 0002:000001e0       __xi_a                     00000001800051e0     MSVCRT:initializers.obj
 0002:000001f0       __xi_z                     00000001800051f0     MSVCRT:initializers.obj
 0002:000001f8       __xl_a                     00000001800051f8     MSVCRT:tlssup.obj
 0002:00000200       __xl_z                     0000000180005200     MSVCRT:tlssup.obj
 0002:00000208       __xp_a                     0000000180005208     MSVCRT:initializers.obj
 0002:00000210       __xp_z                     0000000180005210     MSVCRT:initializers.obj
 0002:00000218       __xt_a                     0000000180005218     MSVCRT:initializers.obj
 0002:00000220       __xt_z                     0000000180005220     MSVCRT:initializers.obj
 0002:00000230       g_refKindStr               0000000180005230     librawmnntfy001.obj
 0002:000003e0       ??_C@_09BPLDFGCI@unknown_0@ 00000001800053e0     librawmnntfy001.obj
 0002:000003f0       ??_C@_0BL@FPNMECJD@JVMTI_HEAP_REFERENCE_CLASS@ 00000001800053f0     librawmnntfy001.obj
 0002:00000410       ??_C@_0BL@FKGKKLNM@JVMTI_HEAP_REFERENCE_FIELD@ 0000000180005410     librawmnntfy001.obj
 0002:00000430       ??_C@_0CD@CAEHCFJF@JVMTI_HEAP_REFERENCE_ARRAY_ELEM@ 0000000180005430     librawmnntfy001.obj
 0002:00000458       ??_C@_0CC@DNEBMCNK@JVMTI_HEAP_REFERENCE_CLASS_LOAD@ 0000000180005458     librawmnntfy001.obj
 0002:00000480       ??_C@_0BN@CJMIPEBB@JVMTI_HEAP_REFERENCE_SIGNERS@ 0000000180005480     librawmnntfy001.obj
 0002:000004a0       ??_C@_0CH@HBOIDPEB@JVMTI_HEAP_REFERENCE_PROTECTION@ 00000001800054a0     librawmnntfy001.obj
 0002:000004c8       ??_C@_0BP@MDKGDGKL@JVMTI_HEAP_REFERENCE_INTERFACE@ 00000001800054c8     librawmnntfy001.obj
 0002:000004e8       ??_C@_0CC@JJMIHNJH@JVMTI_HEAP_REFERENCE_STATIC_FIE@ 00000001800054e8     librawmnntfy001.obj
 0002:00000510       ??_C@_0CD@IDHEEGID@JVMTI_HEAP_REFERENCE_CONSTANT_P@ 0000000180005510     librawmnntfy001.obj
 0002:00000538       ??_C@_0CA@EFFCHNG@JVMTI_HEAP_REFERENCE_SUPERCLASS@ 0000000180005538     librawmnntfy001.obj
 0002:00000558       ??_C@_0L@PCDFHGCJ@unknown_11@ 0000000180005558     librawmnntfy001.obj
 0002:00000568       ??_C@_0L@NJBICFOK@unknown_12@ 0000000180005568     librawmnntfy001.obj
 0002:00000578       ??_C@_0L@MAADBEKL@unknown_13@ 0000000180005578     librawmnntfy001.obj
 0002:00000588       ??_C@_0L@IPECICGM@unknown_14@ 0000000180005588     librawmnntfy001.obj
 0002:00000598       ??_C@_0L@JGFJLDCN@unknown_15@ 0000000180005598     librawmnntfy001.obj
 0002:000005a8       ??_C@_0L@LNHEOAOO@unknown_16@ 00000001800055a8     librawmnntfy001.obj
 0002:000005b8       ??_C@_0L@KEGPNBKP@unknown_17@ 00000001800055b8     librawmnntfy001.obj
 0002:000005c8       ??_C@_0L@CDPHMNGA@unknown_18@ 00000001800055c8     librawmnntfy001.obj
 0002:000005d8       ??_C@_0L@DKOMPMCB@unknown_19@ 00000001800055d8     librawmnntfy001.obj
 0002:000005e8       ??_C@_0L@OJGIPJDB@unknown_20@ 00000001800055e8     librawmnntfy001.obj
 0002:000005f8       ??_C@_0CA@KAOFNDEM@JVMTI_HEAP_REFERENCE_JNI_GLOBAL@ 00000001800055f8     librawmnntfy001.obj
 0002:00000618       ??_C@_0CC@HPFAJBK@JVMTI_HEAP_REFERENCE_SYSTEM_CLA@ 0000000180005618     librawmnntfy001.obj
 0002:00000640       ??_C@_0BN@FDEGFOHC@JVMTI_HEAP_REFERENCE_MONITOR@ 0000000180005640     librawmnntfy001.obj
 0002:00000660       ??_C@_0CB@HKIBCMAJ@JVMTI_HEAP_REFERENCE_STACK_LOCA@ 0000000180005660     librawmnntfy001.obj
 0002:00000688       ??_C@_0BP@EAACMMOE@JVMTI_HEAP_REFERENCE_JNI_LOCAL@ 0000000180005688     librawmnntfy001.obj
 0002:000006a8       ??_C@_0BM@IJDEOGOE@JVMTI_HEAP_REFERENCE_THREAD@ 00000001800056a8     librawmnntfy001.obj
 0002:000006c8       ??_C@_0BL@EDGPPKC@JVMTI_HEAP_REFERENCE_OTHER@ 00000001800056c8     librawmnntfy001.obj
 0002:000006e4       ??_C@_04BCJPDBDA@Code@     00000001800056e4     librawmnntfy001.obj
 0002:000006f0       ??_C@_0BA@OCLMCFKC@LineNumberTable@ 00000001800056f0     librawmnntfy001.obj
 0002:00000700       ??_C@_0BD@CPAEPILC@LocalVariableTable@ 0000000180005700     librawmnntfy001.obj
 0002:00000718       ??_C@_0BH@NMBDNHBD@LocalVariableTypeTable@ 0000000180005718     librawmnntfy001.obj
 0002:00000730       ??_C@_0O@HIHEEDNJ@StackMapTable@ 0000000180005730     librawmnntfy001.obj
 0002:00000740       ??_C@_0L@HCDIAMJG@?9?5?$CFs?0?5?$CFd?3?5@ 0000000180005740     librawmnntfy001.obj
 0002:00000750       ??_C@_0JI@HLPECLFI@?$CD?5?4?4?4?6?$CD?5ERROR?3?5too?5many?5complai@ 0000000180005750     librawmnntfy001.obj
 0002:000007f0       ??_C@_0ED@JNEKCCOB@The?5following?5fake?5exception?5st@ 00000001800057f0     librawmnntfy001.obj
 0002:00000838       ??_C@_0CN@FCNMDFBH@nsk?4share?4Fake_Exception_for_RU@ 0000000180005838     librawmnntfy001.obj
 0002:00000868       ??_C@_08PGFFNAEI@?$CI?$CFs?3?$CFd?$CJ?5@ 0000000180005868     librawmnntfy001.obj
 0002:00000878       ??_C@_0DP@IENMAEGI@s?2test?2hotspot?2jtreg?2vmTestbase@ 0000000180005878     librawmnntfy001.obj
 0002:000008b8       ??_C@_0BL@NDJLFFJB@?7at?5nsk_lvcomplain?$CI?$CFs?3?$CFd?$CJ?6@ 00000001800058b8     librawmnntfy001.obj
 0002:000008d8       ??_C@_0BC@JOOKAFKF@?$CD?5ERROR?3?5?$CFs?0?5?$CFd?3?5@ 00000001800058d8     librawmnntfy001.obj
 0002:000008f0       ??_C@_09KJEAHMEH@?$CD?5ERROR?3?5@ 00000001800058f0     librawmnntfy001.obj
 0002:000008fc       ??_C@_02GPIOPFAK@?$DO?$DO@ 00000001800058fc     librawmnntfy001.obj
 0002:00000900       ??_C@_02FODMEDOG@?$DM?$DM@ 0000000180005900     librawmnntfy001.obj
 0002:00000904       ??_C@_02DJGKEECL@?4?4@     0000000180005904     librawmnntfy001.obj
 0002:00000908       ??_C@_0O@CJPGJOAF@?9?5?$CFs?0?5?$CFd?3?5?$CFs?5@ 0000000180005908     librawmnntfy001.obj
 0002:00000918       ??_C@_0CB@IAKPDOIC@?$CD?5?5?5verified?5assertion?5is?5FALSE@ 0000000180005918     librawmnntfy001.obj
 0002:00000940       ??_C@_0CO@LGONDEPD@stdout?3?5fflush?5failed?5?9?5err?$DN?$CFd?5@ 0000000180005940     librawmnntfy001.obj
 0002:00000970       ??_C@_0CO@KBGKJPBD@stderr?3?5fflush?5failed?5?9?5err?$DN?$CFd?5@ 0000000180005970     librawmnntfy001.obj
 0002:000009a0       ??_C@_0BB@JCNMKLLK@JVMTI_ERROR_NONE@ 00000001800059a0     librawmnntfy001.obj
 0002:000009b8       ??_C@_0BL@LDIMKLPH@JVMTI_ERROR_INVALID_THREAD@ 00000001800059b8     librawmnntfy001.obj
 0002:000009d8       ??_C@_0CB@PJFPAIKJ@JVMTI_ERROR_INVALID_THREAD_GROU@ 00000001800059d8     librawmnntfy001.obj
 0002:00000a00       ??_C@_0BN@LLMKHMNF@JVMTI_ERROR_INVALID_PRIORITY@ 0000000180005a00     librawmnntfy001.obj
 0002:00000a20       ??_C@_0CB@MBOFKAGB@JVMTI_ERROR_THREAD_NOT_SUSPENDE@ 0000000180005a20     librawmnntfy001.obj
 0002:00000a48       ??_C@_0BN@FABOLPBI@JVMTI_ERROR_THREAD_SUSPENDED@ 0000000180005a48     librawmnntfy001.obj
 0002:00000a68       ??_C@_0BN@FDGNOBJM@JVMTI_ERROR_THREAD_NOT_ALIVE@ 0000000180005a68     librawmnntfy001.obj
 0002:00000a88       ??_C@_0BL@GOBIFKNJ@JVMTI_ERROR_INVALID_OBJECT@ 0000000180005a88     librawmnntfy001.obj
 0002:00000aa8       ??_C@_0BK@FCMAJPPC@JVMTI_ERROR_INVALID_CLASS@ 0000000180005aa8     librawmnntfy001.obj
 0002:00000ac8       ??_C@_0BP@IKLLBKEB@JVMTI_ERROR_CLASS_NOT_PREPARED@ 0000000180005ac8     librawmnntfy001.obj
 0002:00000ae8       ??_C@_0BN@KLPPLKG@JVMTI_ERROR_INVALID_METHODID@ 0000000180005ae8     librawmnntfy001.obj
 0002:00000b08       ??_C@_0BN@BCEKOKND@JVMTI_ERROR_INVALID_LOCATION@ 0000000180005b08     librawmnntfy001.obj
 0002:00000b28       ??_C@_0BM@DFDGPME@JVMTI_ERROR_INVALID_FIELDID@ 0000000180005b28     librawmnntfy001.obj
 0002:00000b48       ??_C@_0BL@NELIEPEC@JVMTI_ERROR_NO_MORE_FRAMES@ 0000000180005b48     librawmnntfy001.obj
 0002:00000b68       ??_C@_0BJ@BDBECFDM@JVMTI_ERROR_OPAQUE_FRAME@ 0000000180005b68     librawmnntfy001.obj
 0002:00000b88       ??_C@_0BK@MIIFNLOB@JVMTI_ERROR_TYPE_MISMATCH@ 0000000180005b88     librawmnntfy001.obj
 0002:00000ba8       ??_C@_0BJ@HPCAOILC@JVMTI_ERROR_INVALID_SLOT@ 0000000180005ba8     librawmnntfy001.obj
 0002:00000bc8       ??_C@_0BG@CHILOPNI@JVMTI_ERROR_DUPLICATE@ 0000000180005bc8     librawmnntfy001.obj
 0002:00000be0       ??_C@_0BG@DIEMLHKM@JVMTI_ERROR_NOT_FOUND@ 0000000180005be0     librawmnntfy001.obj
 0002:00000bf8       ??_C@_0BM@NHMCKHOB@JVMTI_ERROR_INVALID_MONITOR@ 0000000180005bf8     librawmnntfy001.obj
 0002:00000c18       ??_C@_0BO@PPEDAJGL@JVMTI_ERROR_NOT_MONITOR_OWNER@ 0000000180005c18     librawmnntfy001.obj
 0002:00000c38       ??_C@_0BG@FCAIPEID@JVMTI_ERROR_INTERRUPT@ 0000000180005c38     librawmnntfy001.obj
 0002:00000c50       ??_C@_0CB@EGDBNKOI@JVMTI_ERROR_INVALID_CLASS_FORMA@ 0000000180005c50     librawmnntfy001.obj
 0002:00000c78       ??_C@_0CG@DGKOGIAL@JVMTI_ERROR_CIRCULAR_CLASS_DEFI@ 0000000180005c78     librawmnntfy001.obj
 0002:00000ca0       ??_C@_0BP@ICEALPKC@JVMTI_ERROR_FAILS_VERIFICATION@ 0000000180005ca0     librawmnntfy001.obj
 0002:00000cc0       ??_C@_0DC@JDACLMIO@JVMTI_ERROR_UNSUPPORTED_REDEFIN@ 0000000180005cc0     librawmnntfy001.obj
 0002:00000cf8       ??_C@_0DE@GKDKNOMJ@JVMTI_ERROR_UNSUPPORTED_REDEFIN@ 0000000180005cf8     librawmnntfy001.obj
 0002:00000d30       ??_C@_0BO@LAFKIOG@JVMTI_ERROR_INVALID_TYPESTATE@ 0000000180005d30     librawmnntfy001.obj
 0002:00000d50       ??_C@_0DH@INDGCLLB@JVMTI_ERROR_UNSUPPORTED_REDEFIN@ 0000000180005d50     librawmnntfy001.obj
 0002:00000d88       ??_C@_0DE@NHEOMMGI@JVMTI_ERROR_UNSUPPORTED_REDEFIN@ 0000000180005d88     librawmnntfy001.obj
 0002:00000dc0       ??_C@_0CA@EKPNJOEP@JVMTI_ERROR_UNSUPPORTED_VERSION@ 0000000180005dc0     librawmnntfy001.obj
 0002:00000de0       ??_C@_0BN@OFFMAHHL@JVMTI_ERROR_NAMES_DONT_MATCH@ 0000000180005de0     librawmnntfy001.obj
 0002:00000e00       ??_C@_0DN@HHBBLAKE@JVMTI_ERROR_UNSUPPORTED_REDEFIN@ 0000000180005e00     librawmnntfy001.obj
 0002:00000e40       ??_C@_0DO@HMBGBGNA@JVMTI_ERROR_UNSUPPORTED_REDEFIN@ 0000000180005e40     librawmnntfy001.obj
 0002:00000e80       ??_C@_0BP@PBECGKHJ@JVMTI_ERROR_UNMODIFIABLE_CLASS@ 0000000180005e80     librawmnntfy001.obj
 0002:00000ea0       ??_C@_0BK@CANILEHF@JVMTI_ERROR_NOT_AVAILABLE@ 0000000180005ea0     librawmnntfy001.obj
 0002:00000ec0       ??_C@_0CE@INJKMEFK@JVMTI_ERROR_MUST_POSSESS_CAPABI@ 0000000180005ec0     librawmnntfy001.obj
 0002:00000ee8       ??_C@_0BJ@LBFPFPDM@JVMTI_ERROR_NULL_POINTER@ 0000000180005ee8     librawmnntfy001.obj
 0002:00000f08       ??_C@_0BP@CHJPNNEM@JVMTI_ERROR_ABSENT_INFORMATION@ 0000000180005f08     librawmnntfy001.obj
 0002:00000f28       ??_C@_0BP@OMFMNLC@JVMTI_ERROR_INVALID_EVENT_TYPE@ 0000000180005f28     librawmnntfy001.obj
 0002:00000f48       ??_C@_0BN@BIBNPHHO@JVMTI_ERROR_ILLEGAL_ARGUMENT@ 0000000180005f48     librawmnntfy001.obj
 0002:00000f68       ??_C@_0BK@KKNDHDCE@JVMTI_ERROR_NATIVE_METHOD@ 0000000180005f68     librawmnntfy001.obj
 0002:00000f88       ??_C@_0BK@PMKCFHAE@JVMTI_ERROR_OUT_OF_MEMORY@ 0000000180005f88     librawmnntfy001.obj
 0002:00000fa8       ??_C@_0BK@NNJBDMNB@JVMTI_ERROR_ACCESS_DENIED@ 0000000180005fa8     librawmnntfy001.obj
 0002:00000fc8       ??_C@_0BI@GHECLMNC@JVMTI_ERROR_WRONG_PHASE@ 0000000180005fc8     librawmnntfy001.obj
 0002:00000fe0       ??_C@_0BF@OLIHJOII@JVMTI_ERROR_INTERNAL@ 0000000180005fe0     librawmnntfy001.obj
 0002:00000ff8       ??_C@_0BO@EOHGKJHI@JVMTI_ERROR_UNATTACHED_THREAD@ 0000000180005ff8     librawmnntfy001.obj
 0002:00001018       ??_C@_0CA@LKHFDACL@JVMTI_ERROR_INVALID_ENVIRONMENT@ 0000000180006018     librawmnntfy001.obj
 0002:00001038       ??_C@_0BA@MMFHLOKK@?$DMunknown?5error?$DO@ 0000000180006038     librawmnntfy001.obj
 0002:00001048       ??_C@_0CF@CBHOKDB@throwable?5?$DN?5jni?9?$DOExceptionOccur@ 0000000180006048     librawmnntfy001.obj
 0002:00001070       ??_C@_03OFAPEBGM@?$CFs?6@  0000000180006070     librawmnntfy001.obj
 0002:00001078       ??_C@_0DM@LPIGEGNJ@s?2test?2hotspot?2jtreg?2vmTestbase@ 0000000180006078     librawmnntfy001.obj
 0002:000010b8       ??_C@_0CC@NFCNPEPK@Exception?5in?5JNI?5call?5?$CIcleared?$CJ@ 00000001800060b8     librawmnntfy001.obj
 0002:000010e0       ??_C@_0BJ@IBAKFIKF@jni?9?$DOExceptionDescribe?$CI?$CJ@ 00000001800060e0     librawmnntfy001.obj
 0002:00001100       ??_C@_0BG@GGKALKMH@jni?9?$DOExceptionClear?$CI?$CJ@ 0000000180006100     librawmnntfy001.obj
 0002:00001118       ??_C@_0CF@JMGFGJLJ@?$CD?5?5?5verified?5JNI?5assertion?5is?5F@ 0000000180006118     librawmnntfy001.obj
 0002:00001140       ??_C@_0CB@MLNJNCLJ@?5?5jvmti?5error?3?5code?$DN?$CFd?0?5name?$DN?$CFs@ 0000000180006140     librawmnntfy001.obj
 0002:00001168       ??_C@_0CD@OHBGDKMK@?$CD?5?5?5jvmti?5error?3?5code?$DN?$CFd?0?5name?$DN@ 0000000180006168     librawmnntfy001.obj
 0002:00001190       ??_C@_0CG@JNNCGPHB@?$CD?5?5?5error?5expected?3?5code?$DN?$CFd?0?5na@ 0000000180006190     librawmnntfy001.obj
 0002:000011c0       ??_C@_0EB@IMGKPCGE@?$CIstr_obj?5?$DN?5jni?9?$DONewStringUTF?$CIco@ 00000001800061c0     librawmnntfy001.obj
 0002:00001210       ??_C@_0EA@HFOGGBCC@s?2test?2hotspot?2jtreg?2vmTestbase@ 0000000180006210     librawmnntfy001.obj
 0002:00001250       ??_C@_05KKCIMGE@error@     0000000180006250     librawmnntfy001.obj
 0002:00001258       ??_C@_0CJ@JACLEAA@Test?5failed?5by?5setFailStatus?$CI?$CJ?4@ 0000000180006258     librawmnntfy001.obj
 0002:00001290       ??_C@_0EA@PNBCDMOA@s?2test?2hotspot?2jtreg?2vmTestbase@ 0000000180006290     librawmnntfy001.obj
 0002:000012d0       ??_C@_0DI@ILAHDLMP@?$CI?$CKagentThreadProc?$CJ?$CIjvmti_env?0?5a@ 00000001800062d0     librawmnntfy001.obj
 0002:00001308       ??_C@_0BD@KDBALNLB@JVMTI?5agent?5thread@ 0000000180006308     librawmnntfy001.obj
 0002:00001320       ??_C@_0BB@NOKBFPFO@java?1lang?1Thread@ 0000000180006320     librawmnntfy001.obj
 0002:00001334       ??_C@_06FALKBLGB@?$DMinit?$DO@ 0000000180006334     librawmnntfy001.obj
 0002:00001340       ??_C@_0BG@IKDDPPGD@?$CILjava?1lang?1String?$DL?$CJV@ 0000000180006340     librawmnntfy001.obj
 0002:00001360       ??_C@_0EB@IFJBFEKC@?$CIthreadClass?5?$DN?5jni_env?9?$DOFindCla@ 0000000180006360     librawmnntfy001.obj
 0002:000013b0       ??_C@_0GF@FGFIBKKL@?$CIthreadCtor?5?$DN?5jni_env?9?$DOGetMetho@ 00000001800063b0     librawmnntfy001.obj
 0002:00001418       ??_C@_0DN@NCPDJLOG@?$CIthreadName?5?$DN?5jni_env?9?$DONewStrin@ 0000000180006418     librawmnntfy001.obj
 0002:00001460       ??_C@_0FE@PFKODBGC@?$CIthreadObject?5?$DN?5jni_env?9?$DONewObj@ 0000000180006460     librawmnntfy001.obj
 0002:000014c0       ??_C@_0ED@HOBAHHJI@?$CIthreadGlobalRef?5?$DN?5jni_env?9?$DONew@ 00000001800064c0     librawmnntfy001.obj
 0002:00001510       ??_C@_0FN@HNJJAHFC@jvmti_env?9?$DORunAgentThread?$CIagent@ 0000000180006510     librawmnntfy001.obj
 0002:00001570       ??_C@_0EA@MOJDNKDF@Debuggee?5status?5sync?5aborted?5be@ 0000000180006570     librawmnntfy001.obj
 0002:000015b0       ??_C@_0EA@EEOEJAEN@status?5?$DN?5syncDebuggeeStatus?$CIjni@ 00000001800065b0     librawmnntfy001.obj
 0002:000015f0       ??_C@_0BL@JBCFNBMB@nsk_jvmti_resetAgentData?$CI?$CJ@ 00000001800065f0     librawmnntfy001.obj
 0002:00001610       ??_C@_0EL@LPBEELIP@s?2test?2hotspot?2jtreg?2vmTestbase@ 0000000180006610     librawmnntfy001.obj
 0002:00001660       ??_C@_0CK@JDAMFDMJ@jvmti?9?$DOSetTag?$CIo?0?5tag?$CJ?5?$DN?$DN?5JVMTI_@ 0000000180006660     librawmnntfy001.obj
 0002:00001690       ??_C@_0CC@DAMNHKNI@Can?8t?5set?5tag?5?$CFli?5for?5object?5?$CFl@ 0000000180006690     librawmnntfy001.obj
 0002:000016b8       ??_C@_0DL@HAJPNKEF@jvmti?9?$DOGetObjectHashCode?$CIo?0?5?$CGha@ 00000001800066b8     librawmnntfy001.obj
 0002:000016f8       ??_C@_0BL@JFPIEOBF@Can?8t?5get?5hash?5object?5?$CFlx?6@ 00000001800066f8     librawmnntfy001.obj
 0002:00001718       ??_C@_0BG@DICPHBKN@setTag?3?5?$CF08x?5?$DM?9?5?$CF?53li@ 0000000180006718     librawmnntfy001.obj
 0002:00001730       ??_C@_0DH@FCEEBDMJ@?$CIs?5?$DN?5jni?9?$DOGetStringUTFChars?$CIsIn@ 0000000180006730     librawmnntfy001.obj
 0002:00001768       ??_C@_0BJ@OKKGHDCN@Can?8t?5get?5string?5at?5?$CF?$CDp?6@ 0000000180006768     librawmnntfy001.obj
 0002:00001788       ??_C@_0BP@EKFLGGFJ@Can?8t?5get?5string?5at?5?$CF?$CDp?3?5null?6@ 0000000180006788     librawmnntfy001.obj
 0002:000017a8       ??_C@_06ICODBHCL@?5?1?1?5?$CFs@ 00000001800067a8     librawmnntfy001.obj
 0002:000017b0       ??_C@_0DB@KGFPLEGO@?$CIr?5?$DN?5jvmti?9?$DOGetTag?$CIo?0?5?$CGtag?$CJ?$CJ?5?$DN?$DN@ 00000001800067b0     librawmnntfy001.obj
 0002:000017e8       ??_C@_0CO@PDAGBCGJ@Can?8t?5GetTag?5for?5object?5?$CFlx?4?5Re@ 00000001800067e8     librawmnntfy001.obj
 0002:00001818       ??_C@_0CH@HPEODOHC@TEST_BUG?3?5Max?4?5number?5of?5refs?5r@ 0000000180006818     librawmnntfy001.obj
 0002:00001840       ??_C@_0DI@PHFCABIM@?$CIr?5?$DN?5jvmti?9?$DOGetTag?$CIfrom?0?5?$CGtagFr@ 0000000180006840     librawmnntfy001.obj
 0002:00001878       ??_C@_0DI@MDEGFNKD@TEST_BUG?3?5Can?8t?5GetTag?5for?5obje@ 0000000180006878     librawmnntfy001.obj
 0002:000018b0       ??_C@_0DE@MLELJAHM@?$CIr?5?$DN?5jvmti?9?$DOGetTag?$CIto?0?5?$CGtagTo?$CJ?$CJ@ 00000001800068b0     librawmnntfy001.obj
 0002:000018e8       ??_C@_0BC@HKHFLNF@?$DO?$DO?$DO?5VMInit?5event?6@ 00000001800068e8     librawmnntfy001.obj
 0002:00001900       ??_C@_0BO@PAAENANI@?$DO?$DO?$DO?5creating?5?$CFd?5raw?5monitors?6@ 0000000180006900     librawmnntfy001.obj
 0002:00001920       ??_C@_0O@CHLKPEI@RawMonitor?9?$CFd@ 0000000180006920     librawmnntfy001.obj
 0002:00001930       ??_C@_0DB@ENBCPHKE@?$CICreateRawMonitor?$CD?$CFd?$CJ?5unexpecte@ 0000000180006930     librawmnntfy001.obj
 0002:00001968       ??_C@_0BO@MMJIBCEC@?$DO?$DO?$DO?5entering?5?$CFd?5raw?5monitors?6@ 0000000180006968     librawmnntfy001.obj
 0002:00001988       ??_C@_0DA@DHIPNKGF@?$CIEnterRawMonitor?$CD?$CFd?$CJ?5unexpected@ 0000000180006988     librawmnntfy001.obj
 0002:000019b8       ??_C@_0BP@MFLOMMKH@?$DO?$DO?$DO?5notifying?5?$CFd?5raw?5monitors?6@ 00000001800069b8     librawmnntfy001.obj
 0002:000019d8       ??_C@_0DB@PFNEPNPK@?$CIRawMonitorNorify?$CD?$CFd?$CJ?5unexpecte@ 00000001800069d8     librawmnntfy001.obj
 0002:00001a10       ??_C@_0BN@BOMNLBKE@?$DO?$DO?$DO?5exiting?5?$CFd?5raw?5monitors?6@ 0000000180006a10     librawmnntfy001.obj
 0002:00001a30       ??_C@_0CP@KDHCBDIM@?$CIRawMonitorExit?$CD?$CFd?$CJ?5unexpected?5@ 0000000180006a30     librawmnntfy001.obj
 0002:00001a60       ??_C@_0CA@CAJLNGOK@?$DO?$DO?$DO?5destroying?5?$CFd?5raw?5monitors?6@ 0000000180006a60     librawmnntfy001.obj
 0002:00001a80       ??_C@_0DC@GGEFDFCH@?$CIDestroyRawMonitor?$CD?$CFd?$CJ?5unexpect@ 0000000180006a80     librawmnntfy001.obj
 0002:00001ab8       ??_C@_09OPJEJKBL@printdump@ 0000000180006ab8     librawmnntfy001.obj
 0002:00001ac8       ??_C@_0CJ@KCDEKOCJ@Wrong?5result?5of?5a?5valid?5call?5to@ 0000000180006ac8     librawmnntfy001.obj
 0002:00001af8       ??_C@_0CP@IMINGNLL@?$CISetEventCallbacks?$CJ?5unexpected?5@ 0000000180006af8     librawmnntfy001.obj
 0002:00001b28       ??_C@_0CP@MDEEHMPF@Failed?5to?5enable?5JVMTI_EVENT_VM@ 0000000180006b28     librawmnntfy001.obj
 0002:00001b58       ??_C@_0BI@MLKNCEPD@?$DO?$DO?$DO?5native?5method?5call?6@ 0000000180006b58     librawmnntfy001.obj
 0002:00001b80       ??_C@_1EC@JIJBPKFM@?$AAa?$AAp?$AAi?$AA?9?$AAm?$AAs?$AA?9?$AAw?$AAi?$AAn?$AA?9?$AAc?$AAo?$AAr?$AAe@ 0000000180006b80     MSVCRT:thread_safe_statics.obj
 0002:00001bc8       ??_C@_1BK@MGMFAEKH@?$AAk?$AAe?$AAr?$AAn?$AAe?$AAl?$AA3?$AA2?$AA?4?$AAd?$AAl?$AAl@ 0000000180006bc8     MSVCRT:thread_safe_statics.obj
 0002:00001be8       ??_C@_0BJ@JEBJOJFJ@SleepConditionVariableCS@ 0000000180006be8     MSVCRT:thread_safe_statics.obj
 0002:00001c08       ??_C@_0BJ@PGPPEPCC@WakeAllConditionVariable@ 0000000180006c08     MSVCRT:thread_safe_statics.obj
 0002:00001c28       _pDefaultRawDllMain        0000000180006c28     MSVCRT:dll_dllmain.obj
 0002:00001c28       _pRawDllMain               0000000180006c28     MSVCRT:dll_dllmain.obj
 0002:00001c30       __xmm@ffffffffffffffffffffffffffffffff 0000000180006c30     MSVCRT:utility.obj
 0002:00001c40       _load_config_used          0000000180006c40     MSVCRT:loadcfg.obj
 0002:00001e00       _tls_used                  0000000180006e00     MSVCRT:tlssup.obj
 0002:00001e28       __volatile_metadata        0000000180006e28     <linker-defined>
 0002:000021e8       __rtc_iaa                  00000001800071e8     MSVCRT:initsect.obj
 0002:000021f0       __rtc_izz                  00000001800071f0     MSVCRT:initsect.obj
 0002:000021f8       __rtc_taa                  00000001800071f8     MSVCRT:initsect.obj
 0002:00002200       __rtc_tzz                  0000000180007200     MSVCRT:initsect.obj
 0002:00002208       _tls_start                 0000000180007208     MSVCRT:tlssup.obj
 0002:0000220c       _Init_thread_epoch         000000018000720c     MSVCRT:thread_safe_statics.obj
 0002:00002210       _tls_end                   0000000180007210     MSVCRT:tlssup.obj
 0002:000028c4       __IMPORT_DESCRIPTOR_KERNEL32 00000001800078c4     kernel32:KERNEL32.dll
 0002:000028d8       __IMPORT_DESCRIPTOR_VCRUNTIME140 00000001800078d8     vcruntime:VCRUNTIME140.dll
 0002:000028ec       __IMPORT_DESCRIPTOR_api-ms-win-crt-runtime-l1-1-0 00000001800078ec     ucrt:api-ms-win-crt-runtime-l1-1-0.dll
 0002:00002900       __IMPORT_DESCRIPTOR_api-ms-win-crt-stdio-l1-1-0 0000000180007900     ucrt:api-ms-win-crt-stdio-l1-1-0.dll
 0002:00002914       __IMPORT_DESCRIPTOR_api-ms-win-crt-string-l1-1-0 0000000180007914     ucrt:api-ms-win-crt-string-l1-1-0.dll
 0002:00002928       __NULL_IMPORT_DESCRIPTOR   0000000180007928     kernel32:KERNEL32.dll
 0003:00000030       _Init_global_epoch         0000000180008030     MSVCRT:thread_safe_statics.obj
 0003:00000040       __security_cookie          0000000180008040     MSVCRT:gs_cookie.obj
 0003:00000048       __security_cookie_complement 0000000180008048     MSVCRT:gs_cookie.obj
 0003:00000050       __scrt_native_dllmain_reason 0000000180008050     MSVCRT:utility.obj
 0003:00000058       __isa_available            0000000180008058     MSVCRT:cpu_disp.obj
 0003:0000005c       __isa_enabled              000000018000805c     MSVCRT:cpu_disp.obj
 0003:00000060       __memset_fast_string_threshold 0000000180008060     MSVCRT:cpu_disp.obj
 0003:00000068       __memset_nt_threshold      0000000180008068     MSVCRT:cpu_disp.obj
 0003:00000070       __scrt_ucrt_dll_is_in_use  0000000180008070     MSVCRT:ucrt_stubs.obj
 0003:00000080       g_wrongHeapCallbacks       0000000180008080     librawmnntfy001.obj
 0003:00000100       g_szTagInfo                0000000180008100     librawmnntfy001.obj
 0003:00002040       g_tagFlags                 000000018000a040     librawmnntfy001.obj
 0003:00002428       g_refsToVerifyCnt          000000018000a428     librawmnntfy001.obj
 0003:0000242c       g_fakeUserData             000000018000a42c     librawmnntfy001.obj
 0003:00002430       g_tagVisitCount            000000018000a430     librawmnntfy001.obj
 0003:000033d0       g_refsToVerify             000000018000b3d0     librawmnntfy001.obj
 0003:0001aad0       g_userDataError            0000000180022ad0     librawmnntfy001.obj
 0003:0001cdb0       ?_OptionsStorage@?1??__local_stdio_printf_options@@9@4_KA 0000000180024db0     librawmnntfy001.obj
 0003:0001d378       _tls_index                 0000000180025378     MSVCRT:tlssup.obj
 0003:0001d380       __scrt_current_native_startup_state 0000000180025380     MSVCRT:utility.obj
 0003:0001d388       __scrt_native_startup_lock 0000000180025388     MSVCRT:utility.obj
 0003:0001d3c8       __scrt_debugger_hook_flag  00000001800253c8     MSVCRT:utility_desktop.obj
 0003:0001d3d0       ?__type_info_root_node@@3U__type_info_node@@A 00000001800253d0     MSVCRT:tncleanup.obj
 0003:0001d3e0       ?_OptionsStorage@?1??__local_stdio_scanf_options@@9@4_KA 00000001800253e0     MSVCRT:default_local_stdio_options.obj
 0003:0001d3e8       __favor                    00000001800253e8     MSVCRT:cpu_disp.obj
 0003:0001d3f0       __dyn_tls_init_callback    00000001800253f0     <common>

 entry point at        0001:000026d0

 Static symbols

 0000:fffd8000       .debug$S                   0000000180000000     rawmnntfy001.exp
 0000:fffd8000       .debug$S                   0000000180000000     vcruntime:VCRUNTIME140.dll
 0000:fffd8000       .debug$S                   0000000180000000     vcruntime:VCRUNTIME140.dll
 0000:fffd8000       .debug$S                   0000000180000000     vcruntime:VCRUNTIME140.dll
 0000:fffd8000       .debug$S                   0000000180000000     vcruntime:VCRUNTIME140.dll
 0000:fffd8000       .debug$S                   0000000180000000     vcruntime:VCRUNTIME140.dll
 0000:fffd8000       .debug$S                   0000000180000000     vcruntime:VCRUNTIME140.dll
 0000:fffd8000       .debug$S                   0000000180000000     vcruntime:VCRUNTIME140.dll
 0000:fffd8000       .debug$S                   0000000180000000     ucrt:api-ms-win-crt-convert-l1-1-0.dll
 0002:ffffb000       .idata$6                   0000000180000000     ucrt:api-ms-win-crt-convert-l1-1-0.dll
 0000:fffd8000       .debug$S                   0000000180000000     ucrt:api-ms-win-crt-heap-l1-1-0.dll
 0000:fffd8000       .debug$S                   0000000180000000     ucrt:api-ms-win-crt-heap-l1-1-0.dll
 0000:fffd8000       .debug$S                   0000000180000000     ucrt:api-ms-win-crt-heap-l1-1-0.dll
 0000:fffd8000       .debug$S                   0000000180000000     ucrt:api-ms-win-crt-heap-l1-1-0.dll
 0002:ffffb000       .idata$6                   0000000180000000     ucrt:api-ms-win-crt-heap-l1-1-0.dll
 0000:fffd8000       .debug$S                   0000000180000000     ucrt:api-ms-win-crt-runtime-l1-1-0.dll
 0000:fffd8000       .debug$S                   0000000180000000     ucrt:api-ms-win-crt-runtime-l1-1-0.dll
 0000:fffd8000       .debug$S                   0000000180000000     ucrt:api-ms-win-crt-runtime-l1-1-0.dll
 0000:fffd8000       .debug$S                   0000000180000000     ucrt:api-ms-win-crt-runtime-l1-1-0.dll
 0000:fffd8000       .debug$S                   0000000180000000     ucrt:api-ms-win-crt-runtime-l1-1-0.dll
 0000:fffd8000       .debug$S                   0000000180000000     ucrt:api-ms-win-crt-runtime-l1-1-0.dll
 0000:fffd8000       .debug$S                   0000000180000000     ucrt:api-ms-win-crt-runtime-l1-1-0.dll
 0000:fffd8000       .debug$S                   0000000180000000     ucrt:api-ms-win-crt-runtime-l1-1-0.dll
 0000:fffd8000       .debug$S                   0000000180000000     ucrt:api-ms-win-crt-runtime-l1-1-0.dll
 0000:fffd8000       .debug$S                   0000000180000000     ucrt:api-ms-win-crt-runtime-l1-1-0.dll
 0000:fffd8000       .debug$S                   0000000180000000     ucrt:api-ms-win-crt-runtime-l1-1-0.dll
 0000:fffd8000       .debug$S                   0000000180000000     ucrt:api-ms-win-crt-runtime-l1-1-0.dll
 0000:fffd8000       .debug$S                   0000000180000000     ucrt:api-ms-win-crt-runtime-l1-1-0.dll
 0000:fffd8000       .debug$S                   0000000180000000     ucrt:api-ms-win-crt-runtime-l1-1-0.dll
 0000:fffd8000       .debug$S                   0000000180000000     ucrt:api-ms-win-crt-runtime-l1-1-0.dll
 0000:fffd8000       .debug$S                   0000000180000000     ucrt:api-ms-win-crt-runtime-l1-1-0.dll
 0000:fffd8000       .debug$S                   0000000180000000     ucrt:api-ms-win-crt-stdio-l1-1-0.dll
 0000:fffd8000       .debug$S                   0000000180000000     ucrt:api-ms-win-crt-stdio-l1-1-0.dll
 0000:fffd8000       .debug$S                   0000000180000000     ucrt:api-ms-win-crt-stdio-l1-1-0.dll
 0000:fffd8000       .debug$S                   0000000180000000     ucrt:api-ms-win-crt-stdio-l1-1-0.dll
 0000:fffd8000       .debug$S                   0000000180000000     ucrt:api-ms-win-crt-stdio-l1-1-0.dll
 0000:fffd8000       .debug$S                   0000000180000000     ucrt:api-ms-win-crt-stdio-l1-1-0.dll
 0000:fffd8000       .debug$S                   0000000180000000     ucrt:api-ms-win-crt-stdio-l1-1-0.dll
 0000:fffd8000       .debug$S                   0000000180000000     ucrt:api-ms-win-crt-stdio-l1-1-0.dll
 0000:fffd8000       .debug$S                   0000000180000000     ucrt:api-ms-win-crt-stdio-l1-1-0.dll
 0000:fffd8000       .debug$S                   0000000180000000     ucrt:api-ms-win-crt-stdio-l1-1-0.dll
 0000:fffd8000       .debug$S                   0000000180000000     ucrt:api-ms-win-crt-string-l1-1-0.dll
 0000:fffd8000       .debug$S                   0000000180000000     ucrt:api-ms-win-crt-string-l1-1-0.dll
 0000:fffd8000       .debug$S                   0000000180000000     ucrt:api-ms-win-crt-string-l1-1-0.dll
 0000:fffd8000       .debug$S                   0000000180000000     ucrt:api-ms-win-crt-string-l1-1-0.dll
 0000:fffd8000       .debug$S                   0000000180000000     ucrt:api-ms-win-crt-string-l1-1-0.dll
 0000:fffd8000       .debug$S                   0000000180000000     ucrt:api-ms-win-crt-string-l1-1-0.dll
 0000:fffd8000       .debug$S                   0000000180000000     ucrt:api-ms-win-crt-string-l1-1-0.dll
 0000:fffd8000       .debug$S                   0000000180000000     ucrt:api-ms-win-crt-string-l1-1-0.dll
 0000:fffd8000       .debug$S                   0000000180000000     kernel32:KERNEL32.dll
 0000:fffd8000       .debug$S                   0000000180000000     kernel32:KERNEL32.dll
 0000:fffd8000       .debug$S                   0000000180000000     kernel32:KERNEL32.dll
 0000:fffd8000       .debug$S                   0000000180000000     kernel32:KERNEL32.dll
 0000:fffd8000       .debug$S                   0000000180000000     kernel32:KERNEL32.dll
 0000:fffd8000       .debug$S                   0000000180000000     kernel32:KERNEL32.dll
 0000:fffd8000       .debug$S                   0000000180000000     kernel32:KERNEL32.dll
 0000:fffd8000       .debug$S                   0000000180000000     kernel32:KERNEL32.dll
 0000:fffd8000       .debug$S                   0000000180000000     kernel32:KERNEL32.dll
 0000:fffd8000       .debug$S                   0000000180000000     kernel32:KERNEL32.dll
 0000:fffd8000       .debug$S                   0000000180000000     kernel32:KERNEL32.dll
 0000:fffd8000       .debug$S                   0000000180000000     kernel32:KERNEL32.dll
 0000:fffd8000       .debug$S                   0000000180000000     kernel32:KERNEL32.dll
 0000:fffd8000       .debug$S                   0000000180000000     kernel32:KERNEL32.dll
 0000:fffd8000       .debug$S                   0000000180000000     kernel32:KERNEL32.dll
 0000:fffd8000       .debug$S                   0000000180000000     kernel32:KERNEL32.dll
 0000:fffd8000       .debug$S                   0000000180000000     kernel32:KERNEL32.dll
 0000:fffd8000       .debug$S                   0000000180000000     kernel32:KERNEL32.dll
 0000:fffd8000       .debug$S                   0000000180000000     kernel32:KERNEL32.dll
 0000:fffd8000       .debug$S                   0000000180000000     kernel32:KERNEL32.dll
 0000:fffd8000       .debug$S                   0000000180000000     kernel32:KERNEL32.dll
 0000:fffd8000       .debug$S                   0000000180000000     kernel32:KERNEL32.dll
 0000:fffd8000       .debug$S                   0000000180000000     kernel32:KERNEL32.dll
 0000:fffd8000       .debug$S                   0000000180000000     kernel32:KERNEL32.dll
 0000:fffd8000       .debug$S                   0000000180000000     kernel32:KERNEL32.dll
 0000:fffd8000       .debug$S                   0000000180000000     kernel32:KERNEL32.dll
 0000:fffd8000       .debug$S                   0000000180000000     kernel32:KERNEL32.dll
 0000:fffd8000       .debug$S                   0000000180000000     kernel32:KERNEL32.dll
 0001:000012f0       addRefToVerify             00000001800022f0 f   librawmnntfy001.obj
 0001:0000135c       agentThreadWrapper         000000018000235c f   librawmnntfy001.obj
 0001:0000154c       file_basename              000000018000254c f   librawmnntfy001.obj
 0001:00001bb8       startAgentThreadWrapper    0000000180002bb8 f   librawmnntfy001.obj
 0001:00001ef8       syncDebuggeeStatus         0000000180002ef8 f   librawmnntfy001.obj
 0001:00002198       capture_previous_context   0000000180003198 f   MSVCRT:gs_report.obj
 0001:0000220c       ?__scrt_initialize_thread_safe_statics@@YAHXZ 000000018000320c f   MSVCRT:thread_safe_statics.obj
 0001:000022dc       ?__scrt_uninitialize_thread_safe_statics@@YAXXZ 00000001800032dc f   MSVCRT:thread_safe_statics.obj
 0001:00002380       $$000000                   0000000180003380     MSVCRT:amdsecgs.obj
 0001:000023b0       ?dllmain_crt_dispatch@@YAHQEAUHINSTANCE__@@KQEAX@Z 00000001800033b0 f   MSVCRT:dll_dllmain.obj
 0001:00002400       ?dllmain_crt_process_attach@@YAHQEAUHINSTANCE__@@QEAX@Z 0000000180003400 f   MSVCRT:dll_dllmain.obj
 0001:00002518       ?dllmain_crt_process_detach@@YAH_N@Z 0000000180003518 f   MSVCRT:dll_dllmain.obj
 0001:0000259c       ?dllmain_dispatch@@YAHQEAUHINSTANCE__@@KQEAX@Z 000000018000359c f   MSVCRT:dll_dllmain.obj
 0001:00002fb0       $$000000                   0000000180003fb0     MSVCRT:guard_dispatch.obj
 0001:00002fd0       $$000000                   0000000180003fd0     MSVCRT:guard_xfg_dispatch.obj
 0001:00002fe6       ?fin$0@?0??dllmain_crt_process_attach@@YAHQEAUHINSTANCE__@@QEAX@Z@4HA 0000000180003fe6 f   MSVCRT:dll_dllmain.obj
 0001:00002ffd       ?fin$0@?0??dllmain_crt_process_detach@@YAH_N@Z@4HA 0000000180003ffd f   MSVCRT:dll_dllmain.obj
 0001:00003016       ?fin$1@?0??dllmain_crt_process_detach@@YAH_N@Z@4HA 0000000180004016 f   MSVCRT:dll_dllmain.obj
 0001:0000302a       ?filt$0@?0??dllmain_dispatch@@YAHQEAUHINSTANCE__@@KQEAX@Z@4HA 000000018000402a f   MSVCRT:dll_dllmain.obj
 0001:00003060       __scrt_is_nonwritable_in_current_image$filt$0 0000000180004060 f   MSVCRT:utility.obj
 0002:000001e8       ?__scrt_initialize_tss_var@@3P6AHXZEA 00000001800051e8     MSVCRT:thread_safe_statics.obj
 0002:00000310       ?opcLengths@@3QBEB         0000000180005310     librawmnntfy001.obj
 0002:00001b70       GS_ExceptionPointers       0000000180006b70     MSVCRT:gs_report.obj
 0002:00002218       $unwind$fprintf            0000000180007218     librawmnntfy001.obj
 0002:00002224       $unwind$printf             0000000180007224     librawmnntfy001.obj
 0002:00002230       $unwind$_snprintf          0000000180007230     librawmnntfy001.obj
 0002:00002240       $unwind$?NewObject@JNIEnv_@@QEAAPEAV_jobject@@PEAV_jclass@@PEAU_jmethodID@@ZZ 0000000180007240     librawmnntfy001.obj
 0002:00002240       $unwind$nsk_lcomplain      0000000180007240     librawmnntfy001.obj
 0002:00002240       $unwind$nsk_ldisplay       0000000180007240     librawmnntfy001.obj
 0002:00002248       $unwind$Agent_Initialize   0000000180007248     librawmnntfy001.obj
 0002:00002248       $unwind$nsk_lvdisplay      0000000180007248     librawmnntfy001.obj
 0002:00002248       $unwind$_RTC_Initialize    0000000180007248     MSVCRT:initsect.obj
 0002:00002248       $unwind$_RTC_Terminate     0000000180007248     MSVCRT:initsect.obj
 0002:00002248       $unwind$?__scrt_initialize_thread_safe_statics@@YAHXZ 0000000180007248     MSVCRT:thread_safe_statics.obj
 0002:00002254       $unwind$nsk_lvcomplain     0000000180007254     librawmnntfy001.obj
 0002:0000226c       $unwind$nsk_ltrace         000000018000726c     librawmnntfy001.obj
 0002:0000226c       $unwind$__report_gsfailure 000000018000726c     MSVCRT:gs_report.obj
 0002:00002274       $unwind$nsk_lvtrace        0000000180007274     librawmnntfy001.obj
 0002:00002274       $unwind$__raise_securityfailure 0000000180007274     MSVCRT:gs_report.obj
 0002:00002274       $unwind$__scrt_initialize_crt 0000000180007274     MSVCRT:utility.obj
 0002:00002274       $unwind$__scrt_initialize_onexit_tables 0000000180007274     MSVCRT:utility.obj
 0002:00002274       $unwind$__scrt_release_startup_lock 0000000180007274     MSVCRT:utility.obj
 0002:00002274       $unwind$__scrt_uninitialize_crt 0000000180007274     MSVCRT:utility.obj
 0002:00002274       $unwind$_onexit            0000000180007274     MSVCRT:utility.obj
 0002:0000227c       $unwind$nsk_lverify        000000018000727c     librawmnntfy001.obj
 0002:0000228c       $unwind$nsk_vprintf        000000018000728c     librawmnntfy001.obj
 0002:0000229c       $unwind$nsk_printf         000000018000729c     librawmnntfy001.obj
 0002:000022a4       $unwind$?nsk_jni_lverify@@YAHHPEAUJNIEnv_@@HQEBDH1ZZ 00000001800072a4     librawmnntfy001.obj
 0002:000022b8       $unwind$?nsk_jni_check_exception@@YAHPEAUJNIEnv_@@QEBDH@Z 00000001800072b8     librawmnntfy001.obj
 0002:000022d4       $unwind$Java_nsk_jvmti_unit_FollowReferences_FollowRefObjects_resetTags 00000001800072d4     librawmnntfy001.obj
 0002:000022d4       $unwind$addRefToVerify     00000001800072d4     librawmnntfy001.obj
 0002:000022d4       $unwind$nsk_jvmti_resetAgentData 00000001800072d4     librawmnntfy001.obj
 0002:000022d4       $unwind$nsk_jvmti_setFailStatus 00000001800072d4     librawmnntfy001.obj
 0002:000022d4       $unwind$__scrt_initialize_default_local_stdio_options 00000001800072d4     MSVCRT:default_local_stdio_options.obj
 0002:000022d4       $unwind$?dllmain_crt_dispatch@@YAHQEAUHINSTANCE__@@KQEAX@Z 00000001800072d4     MSVCRT:dll_dllmain.obj
 0002:000022d4       $unwind$DllMain            00000001800072d4     MSVCRT:dll_dllmain_stub.obj
 0002:000022d4       $unwind$__GSHandlerCheck   00000001800072d4     MSVCRT:gshandler.obj
 0002:000022d4       $unwind$?__scrt_uninitialize_thread_safe_statics@@YAXXZ 00000001800072d4     MSVCRT:thread_safe_statics.obj
 0002:000022d4       $unwind$__scrt_acquire_startup_lock 00000001800072d4     MSVCRT:utility.obj
 0002:000022d4       $unwind$__scrt_dllmain_after_initialize_c 00000001800072d4     MSVCRT:utility.obj
 0002:000022d4       $unwind$__scrt_dllmain_before_initialize_c 00000001800072d4     MSVCRT:utility.obj
 0002:000022d4       $unwind$__scrt_dllmain_crt_thread_attach 00000001800072d4     MSVCRT:utility.obj
 0002:000022d4       $unwind$__scrt_dllmain_crt_thread_detach 00000001800072d4     MSVCRT:utility.obj
 0002:000022d4       $unwind$__scrt_dllmain_uninitialize_c 00000001800072d4     MSVCRT:utility.obj
 0002:000022d4       $unwind$__scrt_dllmain_uninitialize_critical 00000001800072d4     MSVCRT:utility.obj
 0002:000022d4       $unwind$atexit             00000001800072d4     MSVCRT:utility.obj
 0002:000022dc       $unwind$nsk_jvmti_lverify  00000001800072dc     librawmnntfy001.obj
 0002:000022f0       $unwind$exitOnError        00000001800072f0     librawmnntfy001.obj
 0002:00002300       $unwind$Java_nsk_share_jvmti_ArgumentHandler_getAgentOptionsString 0000000180007300     librawmnntfy001.obj
 0002:00002314       $unwind$Java_nsk_jvmti_unit_FollowReferences_FollowRefObjects_getTag 0000000180007314     librawmnntfy001.obj
 0002:00002314       $unwind$Java_nsk_share_jvmti_DebugeeClass_checkStatus 0000000180007314     librawmnntfy001.obj
 0002:00002314       $unwind$agentThreadWrapper 0000000180007314     librawmnntfy001.obj
 0002:00002324       $unwind$startAgentThreadWrapper 0000000180007324     librawmnntfy001.obj
 0002:00002340       $unwind$syncDebuggeeStatus 0000000180007340     librawmnntfy001.obj
 0002:00002340       $unwind$__scrt_dllmain_exception_filter 0000000180007340     MSVCRT:utility.obj
 0002:00002354       $unwind$Java_nsk_share_jvmti_DebugeeClass_resetAgentData 0000000180007354     librawmnntfy001.obj
 0002:0000235c       $unwind$MA_checkStatus     000000018000735c     librawmnntfy001.obj
 0002:00002370       $unwind$Java_nsk_jvmti_unit_FollowReferences_FollowRefObjects_setTag 0000000180007370     librawmnntfy001.obj
 0002:00002388       $unwind$Java_nsk_jvmti_unit_FollowReferences_FollowRefObjects_addRefToVerify 0000000180007388     librawmnntfy001.obj
 0002:000023a4       $unwind$Java_nsk_jvmti_RawMonitorNotify_rawmnntfy001_check 00000001800073a4     librawmnntfy001.obj
 0002:000023a4       $unwind$VMInit             00000001800073a4     librawmnntfy001.obj
 0002:000023c4       $unwind$capture_previous_context 00000001800073c4     MSVCRT:gs_report.obj
 0002:000023d0       $unwind$__GSHandlerCheckCommon 00000001800073d0     MSVCRT:gshandler.obj
 0002:000023d8       $xdatasym                  00000001800073d8     MSVCRT:amdsecgs.obj
 0002:000023dc       $unwind$?dllmain_crt_process_attach@@YAHQEAUHINSTANCE__@@QEAX@Z 00000001800073dc     MSVCRT:dll_dllmain.obj
 0002:00002418       $unwind$?fin$0@?0??dllmain_crt_process_attach@@YAHQEAUHINSTANCE__@@QEAX@Z@4HA 0000000180007418     MSVCRT:dll_dllmain.obj
 0002:00002418       $unwind$?fin$0@?0??dllmain_crt_process_detach@@YAH_N@Z@4HA 0000000180007418     MSVCRT:dll_dllmain.obj
 0002:00002418       $unwind$?fin$1@?0??dllmain_crt_process_detach@@YAH_N@Z@4HA 0000000180007418     MSVCRT:dll_dllmain.obj
 0002:00002420       $unwind$?dllmain_crt_process_detach@@YAH_N@Z 0000000180007420     MSVCRT:dll_dllmain.obj
 0002:00002474       $unwind$?dllmain_dispatch@@YAHQEAUHINSTANCE__@@KQEAX@Z 0000000180007474     MSVCRT:dll_dllmain.obj
 0002:0000249c       $unwind$?filt$0@?0??dllmain_dispatch@@YAHQEAUHINSTANCE__@@KQEAX@Z@4HA 000000018000749c     MSVCRT:dll_dllmain.obj
 0002:000024a4       $unwind$_DllMainCRTStartup 00000001800074a4     MSVCRT:dll_dllmain.obj
 0002:000024b4       $unwind$__scrt_is_nonwritable_in_current_image 00000001800074b4     MSVCRT:utility.obj
 0002:000024d4       $unwind$__scrt_is_nonwritable_in_current_image$filt$0 00000001800074d4     MSVCRT:utility.obj
 0002:000024dc       $unwind$__scrt_fastfail    00000001800074dc     MSVCRT:utility_desktop.obj
 0002:000024ec       $unwind$__security_init_cookie 00000001800074ec     MSVCRT:gs_support.obj
 0002:000024f8       $unwind$__isa_available_init 00000001800074f8     MSVCRT:cpu_disp.obj
 0002:00002508       $xdatasym                  0000000180007508     MSVCRT:guard_dispatch.obj
 0002:00002510       $xdatasym                  0000000180007510     MSVCRT:guard_xfg_dispatch.obj
 0002:00002520       .edata                     0000000180007520     rawmnntfy001.exp
 0002:00002548       rgpv                       0000000180007548     rawmnntfy001.exp
 0002:00002584       rgszName                   0000000180007584     rawmnntfy001.exp
 0002:000025c0       rgwOrd                     00000001800075c0     rawmnntfy001.exp
 0002:000025de       szName                     00000001800075de     rawmnntfy001.exp
 0002:000025ef       $N00001                    00000001800075ef     rawmnntfy001.exp
 0002:000025fe       $N00002                    00000001800075fe     rawmnntfy001.exp
 0002:0000260b       $N00003                    000000018000760b     rawmnntfy001.exp
 0002:0000263e       $N00004                    000000018000763e     rawmnntfy001.exp
 0002:00002683       $N00005                    0000000180007683     rawmnntfy001.exp
 0002:000026c0       $N00006                    00000001800076c0     rawmnntfy001.exp
 0002:00002708       $N00007                    0000000180007708     rawmnntfy001.exp
 0002:00002748       $N00008                    0000000180007748     rawmnntfy001.exp
 0002:00002785       $N00009                    0000000180007785     rawmnntfy001.exp
 0002:000027c0       $N00010                    00000001800077c0     rawmnntfy001.exp
 0002:000027ee       $N00011                    00000001800077ee     rawmnntfy001.exp
 0002:0000281f       $N00012                    000000018000781f     rawmnntfy001.exp
 0002:0000284e       $N00013                    000000018000784e     rawmnntfy001.exp
 0002:0000287d       $N00014                    000000018000787d     rawmnntfy001.exp
 0002:000028b2       $N00015                    00000001800078b2     rawmnntfy001.exp
 0002:00002cc2       .idata$6                   0000000180007cc2     kernel32:KERNEL32.dll
 0002:00002d26       .idata$6                   0000000180007d26     vcruntime:VCRUNTIME140.dll
 0002:00002e92       .idata$6                   0000000180007e92     ucrt:api-ms-win-crt-runtime-l1-1-0.dll
 0002:00002eb4       .idata$6                   0000000180007eb4     ucrt:api-ms-win-crt-stdio-l1-1-0.dll
 0002:00002ed4       .idata$6                   0000000180007ed4     ucrt:api-ms-win-crt-string-l1-1-0.dll
 0003:00000000       ?codeAttributeName@@3PEBDEB 0000000180008000     librawmnntfy001.obj
 0003:00000008       ?lineNumberAttributeName@@3PEBDEB 0000000180008008     librawmnntfy001.obj
 0003:00000010       ?localVarAttributeName@@3PEBDEB 0000000180008010     librawmnntfy001.obj
 0003:00000018       ?localVarTypeAttributeName@@3PEBDEB 0000000180008018     librawmnntfy001.obj
 0003:00000020       ?stackMapAttributeName@@3PEBDEB 0000000180008020     librawmnntfy001.obj
 0003:00000028       ?callBytes@@3PAEA          0000000180008028     librawmnntfy001.obj
 0003:0000002c       ?allocBytes@@3PAEA         000000018000802c     librawmnntfy001.obj
 0003:0001aad4       redefineAttempted          0000000180022ad4     librawmnntfy001.obj
 0003:0001aad8       nsk_context                0000000180022ad8     librawmnntfy001.obj
 0003:0001aae4       redefineSucceed            0000000180022ae4     librawmnntfy001.obj
 0003:0001aae8       agentFailed                0000000180022ae8     librawmnntfy001.obj
 0003:0001aaec       currentAgentStatus         0000000180022aec     librawmnntfy001.obj
 0003:0001aaf0       context                    0000000180022af0     librawmnntfy001.obj
 0003:0001aba8       agentThread                0000000180022ba8     librawmnntfy001.obj
 0003:0001abb0       agentThreadProc            0000000180022bb0     librawmnntfy001.obj
 0003:0001abb8       agentThreadArg             0000000180022bb8     librawmnntfy001.obj
 0003:0001abc0       agent_data                 0000000180022bc0     librawmnntfy001.obj
 0003:0001abd0       jvmti_env                  0000000180022bd0     librawmnntfy001.obj
 0003:0001abd8       jvm                        0000000180022bd8     librawmnntfy001.obj
 0003:0001abe0       jni_env                    0000000180022be0     librawmnntfy001.obj
 0003:0001abe8       checkStatus_func           0000000180022be8     librawmnntfy001.obj
 0003:0001abf0       ?codeAttributeIndex@@3GA   0000000180022bf0     librawmnntfy001.obj
 0003:0001abf2       printdump                  0000000180022bf2     librawmnntfy001.obj
 0003:0001abf4       ?lineNumberAttributeIndex@@3GA 0000000180022bf4     librawmnntfy001.obj
 0003:0001abf8       ?localVarAttributeIndex@@3GA 0000000180022bf8     librawmnntfy001.obj
 0003:0001abfc       ?localVarTypeAttributeIndex@@3GA 0000000180022bfc     librawmnntfy001.obj
 0003:0001ac00       ?stackMapAttributeIndex@@3GA 0000000180022c00     librawmnntfy001.obj
 0003:0001ac04       ?stackFrameOffset@@3GA     0000000180022c04     librawmnntfy001.obj
 0003:0001ac08       ?mode@@3HA                 0000000180022c08     librawmnntfy001.obj
 0003:0001ac0c       ?constantPoolSize@@3GA     0000000180022c0c     librawmnntfy001.obj
 0003:0001ac10       ?orig@@3PEBEEB             0000000180022c10     librawmnntfy001.obj
 0003:0001ac18       ?gen@@3PEAEEA              0000000180022c18     librawmnntfy001.obj
 0003:0001ac20       ?inputPos@@3PEAEEA         0000000180022c20     librawmnntfy001.obj
 0003:0001ac28       ?endPos@@3PEBEEB           0000000180022c28     librawmnntfy001.obj
 0003:0001ac30       ?genPos@@3PEAEEA           0000000180022c30     librawmnntfy001.obj
 0003:0001ac38       ?markPos@@3PEAEEA          0000000180022c38     librawmnntfy001.obj
 0003:0001ac40       ?constantPool@@3PEAPEADEA  0000000180022c40     librawmnntfy001.obj
 0003:0001ac48       ?constantPoolCount@@3GA    0000000180022c48     librawmnntfy001.obj
 0003:0001ac4c       ?zeroBytes@@3PAEA          0000000180022c4c     librawmnntfy001.obj
 0003:0001ac50       ?codeLength@@3IA           0000000180022c50     librawmnntfy001.obj
 0003:0001ac54       result                     0000000180022c54     librawmnntfy001.obj
 0003:0001ac58       ?map@@3PEAIEA              0000000180022c58     librawmnntfy001.obj
 0003:0001ac60       ?widening@@3PEACEA         0000000180022c60     librawmnntfy001.obj
 0003:0001ac68       jvmti                      0000000180022c68     librawmnntfy001.obj
 0003:0001ac70       callbacks                  0000000180022c70     librawmnntfy001.obj
 0003:0001adb0       monitors                   0000000180022db0     librawmnntfy001.obj
 0003:0001cdc0       GS_ExceptionRecord         0000000180024dc0     MSVCRT:gs_report.obj
 0003:0001ce60       GS_ContextRecord           0000000180024e60     MSVCRT:gs_report.obj
 0003:0001d330       ?g_tss_cv@@3U_RTL_CONDITION_VARIABLE@@A 0000000180025330     MSVCRT:thread_safe_statics.obj
 0003:0001d338       ?g_tss_event@@3PEAXEA      0000000180025338     MSVCRT:thread_safe_statics.obj
 0003:0001d340       ?g_tss_mutex@@3U_RTL_CRITICAL_SECTION@@A 0000000180025340     MSVCRT:thread_safe_statics.obj
 0003:0001d368       ?g_sleep_condition_variable_cs@@3P6AHPEAU_RTL_CONDITION_VARIABLE@@PEAU_RTL_CRITICAL_SECTION@@K@ZEA 0000000180025368     MSVCRT:thread_safe_statics.obj
 0003:0001d370       ?g_wake_all_condition_variable@@3P6AXPEAU_RTL_CONDITION_VARIABLE@@@ZEA 0000000180025370     MSVCRT:thread_safe_statics.obj
 0003:0001d37c       ?__proc_attached@@3HA      000000018002537c     MSVCRT:dll_dllmain.obj
 0003:0001d390       ?is_initialized_as_dll@@3_NA 0000000180025390     MSVCRT:utility.obj
 0003:0001d391       ?module_local_atexit_table_initialized@@3_NA 0000000180025391     MSVCRT:utility.obj
 0003:0001d398       ?module_local_atexit_table@@3U_onexit_table_t@@A 0000000180025398     MSVCRT:utility.obj
 0003:0001d3b0       ?module_local_at_quick_exit_table@@3U_onexit_table_t@@A 00000001800253b0     MSVCRT:utility.obj
